:10000000020587C0E0C0D075D000C000781806E6B1
:1000100018700106C2CFD000D0D0D0E03202170055
:020020000000DE
:03002300020613BF
:10002B00020003E4F52DF5347535FF753625F537EC
:10003B00F538F539F53A1206F67BFF7A07797E1219
:10004B0007EA7BFF7A0779911207EAC297D290E40D
:10005B007817F608F6C37818E6942818E69400404B
:10006B00F4D2977BFF7A0779A41207EA12088AC2A7
:10007B00FFE4F5A375ECFF12087BD3EF9400EE942D
:10008B0000400543340880035334F77817E6FE0825
:10009B00E6FF65387003EE6537600C8E378F3805D9
:1000AB003AE53A70020539C3EF9450EE94004006DE
:1000BB00E47817F608F6C3E53A94C8E5399400409E
:1000CB000F753900753AC8D290D2975334CF801E32
:1000DB00C3E53A9464E53994004007D2975334EF63
:1000EB00800CE53430E407C29730E502C2908534CA
:1000FB003530FF80C2FF85A321E52DB40E004003F0
:10010B00020324900115F828287302013F02017E97
:10011B000201870201990201AC0202A3020324022D
:10012B00030002030202031502021F02022902024C
:10013B002F020263E52124AB601B24B2601D146007
:10014B002014602924FB601F2450600302007F757C
:10015B002D0102007F752D0402007F752D09020011
:10016B007F8536A302007F752D0802007F8534A39F
:10017B0002031E85212E752D0202007F85212FE59E
:10018B002F7005F52D02007F752D0302007FAF2127
:10019B001204E3152FE52F600302007FF52D0200FB
:1001AB007F85212E12087B8E308F31D3EF9400EE9A
:1001BB0094004058D3E5319408E53094004006751F
:1001CB003000753108AF31EFF5A3E4F522E52E646D
:1001DB000270338F22F532F533F521E521C39522D9
:1001EB00501E12068E74242521F8A607742425218F
:1001FB00F8E67E002533FF7532008F33052180DB57
:10020B00752D0A02007F752D0502007FE4F5A3F51D
:10021B002D02007FE522F4F5A3E4F5238034752D40
:10022B000C02007FE521B4060302031EE521B4187E
:10023B001BE4F521E521C39522500E74242521F8EA
:10024B00E6FF12080F052180EB02031E8524A37520
:10025B002301752D0D02007FE521B4181BE4F52158
:10026B00E521C39522500E74242521F8E6FF1208D0
:10027B000F052180EB02031EE523C39522500EAF21
:10028B0023052374242FF8E6F5A302007FE533F44E
:10029B00F5A3752D0B02007FE521B4181AE4F521A7
:1002AB00E521C39522500E74242521F8E6FF120890
:1002BB000F052180EB805CD3E5319400E530940091
:1002CB00403112068E8F218521A3AF220522742483
:1002DB002FF8A621E522C394094003752208E531C6
:1002EB00153170021530144530600302007FF52D77
:1002FB0002007F801E801C5334F8E52154374234B2
:10030B00E4F539F53AF52D02007FAF211204398F50
:10031B00368FA3E4F52D02007FE4F52D02007FE775
:10032B0009F608DFFA8046E709F208DFFA803E8813
:10033B00828C83E709F0A3DFFA8032E309F608DF4A
:10034B00FA8078E309F208DFFA807088828C83E305
:10035B0009F0A3DFFA806489828A83E0A3F608DFC1
:10036B00FA805889828A83E0A3F208DFFA804C80F6
:10037B00D280FA80C680D4806980F280338010806E
:10038B00A680EA809A80A880DA80E280CA803389CE
:10039B00828A83ECFAE493A3C8C582C8CCC583CC0C
:1003AB00F0A3C8C582C8CCC583CCDFE9DEE7800DDE
:1003BB0089828A83E493A3F608DFF9ECFAA9F0EDBE
:1003CB00FB2289828A83ECFAE0A3C8C582C8CCC51C
:1003DB0083CCF0A3C8C582C8CCC583CCDFEADEE8EA
:1003EB0080DB89828A83E493A3F208DFF980CC88CF
:1003FB00F0EF60010E4E60C388F0ED2402B40400F0
:10040B0050B9F582EB2402B4040050AF232345828C
:10041B002390037A73BB010689828A83E022500200
:10042B00E722BBFE02E32289828A83E493228F3C7C
:10043B00538EF4E53CC39425404DC2CA75B2837507
:10044B00CB9C75CA4FD2CAE53C24C8601624ED601C
:10045B001724DB601824DA601924B5601A24BC70E9
:10046B001E801F758DB8806D758DCB8068758D96D0
:10047B008056758DB08051758D2B438E08805675C7
:10048B003C25758D96804EC2CA75B28075CB3C7576
:10049B00CAB0D2CAE53C24FE601924FE601D24FBC1
:1004AB00601E24F7601F24ED602324247021758DBA
:1004BB00968003758DCB438E02801A758D6A8015DD
:1004CB00758D608003758DB0438E01800880037538
:1004DB003C25758DA0AF3C228F3FD37816E6940058
:1004EB0018E694004058D2017815E6FE08E6FF782E
:1004FB0013E6FC08E6FDD39FEC9E5009E408F608D2
:10050B00F678138034C3EF944BEE9400402EED78C5
:10051B0016967914F7EC189619F77813E6FE08E699
:10052B00FF7816E62442F9E43401FA7B0178427C29
:10053B00017D011203FAE47815F608F6C201C378BF
:10054B0014E6949518E6940040107816E618467059
:10055B00953002F6C202D29980F078130806E6189D
:10056B008606700106142442F58274013EF583E57C
:10057B003FF0300204C202D299AF3F22787FE4F6FB
:10058B00D8FD75813F0205CE02002EE493A3F8E45B
:10059B0093A34003F68001F208DFF48029E493A3D0
:1005AB00F85407240CC8C333C4540F4420C88340E9
:1005BB0004F456800146F6DFE4800B0102040810B8
:1005CB0020408090001DE47E019360BCA3FF543F4C
:1005DB0030E509541FFEE493A360010ECF54C025F0
:1005EB00E060A840B8E493A3FAE493A3F8E493A3E0
:1005FB00C8C582C8CAC583CAF0A3C8C582C8CAC544
:10060B0083CADFE9DEE780BEC0E0C083C082C0D012
:10061B0075D00830982FC298C37812E6943F18E62D
:10062B00940150150806E618860E70010614240175
:10063B00F58274003EF5838009C292C294C29390F6
:10064B000000E599F0309932C29920012BD379142F
:10065B00E778169619E7189640180806E618860EDE
:10066B00700106142442F58274013EF583E0F5997E
:10067B008002D202D2008002D202D0D0D082D083AC
:10068B00D0E0327812E6184670099001D9E0700379
:10069B007FFF229001D9E0601EA3E0F53B9001D9CA
:1006AB00E014F0603DE0FF7E0078DA7C017D017B99
:1006BB00017A0179DB8028900001E0F53B78110885
:1006CB00E616187001161486064E60167811E6FEB3
:1006DB0008E6FF78017C007D017B017A007902122C
:1006EB0003FAD292D294D293AF3B2253D9BFE4F503
:1006FB00A8F5B8F5E6F5F675E477D2971208837589
:10070B00D90275EBFF75ECFF12086B120829120862
:10071B0042120740E4F53B120859053BE53BC394F5
:10072B006440F4D2AFE4F53B120859053BE53BC3FB
:10073B00946440F422C299C28EC2AB759810D29CBD
:10074B007F25120439758BFF53890F438920D20003
:10075B00D202C201E47811F608F69001D9F008F63E
:10076B0008F608F608F6C299C298D2ACD2BCD29958
:10077B00D28E22202020202020202020202020204C
:10078B002020200D0A004E4F41412033333120539E
:10079B007461727475700D0A004E4F4141203333F2
:1007AB0031204C6F6F700D0A008F3EE53ED3947F66
:1007BB0040037F0022E53EB40A057F0D1204E3E5FA
:1007CB003EC394205011E53E24F824FD500924FE2D
:1007DB00600580007F0022AF3E1204E3AF3E228B08
:1007EB003B8A3C893DAB3BAA3CA93D1204206013DC
:1007FB00053DE53D7002053C14F9120420FF12077C
:10080B00B480E2229001D9E0C394135010E0FE04AF
:10081B00F074DA2EF582E43401F583EFF02275A43F
:10082B005475A5F475F1FF75F2FFE4F5D475D5FF9A
:10083B0075E10B75E24022E4F5C8538ECF75CB9E64
:10084B0075CA5874FFF5CDF5CCD2ADD2CA22E4FFF0
:10085B00FE75ECFF0FBF00010EBE01F5BFF4F222D7
:10086B0075A20B75A10775F804D2F9D2F8C2FF2255
:10087B007811E6FE08E6FF22E4F5A975B28322E4BF
:06088B007811F608F622C8
:00000001FF
